:1000000018F09FE518F09FE518F09FE518F09FE5C0
:1000100018F09FE5606FA0B814F09FE514F09FE51D
:1000200010040000FC0400000005000004050000AE
:1000300008050000800500000C050000000000001D
:1000400000000000000000000000000000000000B0
:1000500000000000000000000000000000000000A0
:100060000000000000000000000000000000000090
:100070000000000000000000000000000000000080
:100080000000000000000000000000000000000070
:100090000000000000000000000000000000000060
:1000A0000000000000000000000000000000000050
:1000B0000000000000000000000000000000000040
:1000C0000000000000000000000000000000000030
:1000D0000000000000000000000000000000000020
:1000E0000000000000000000000000000000000010
:1000F0000000000000000000000000000000000000
:1001000000000000000000000000000000000000EF
:1001100000000000000000000000000000000000DF
:1001200000000000000000000000000000000000CF
:1001300000000000000000000000000000000000BF
:1001400000000000000000000000000000000000AF
:10015000000000000000000000000000000000009F
:10016000000000000000000000000000000000008F
:10017000000000000000000000000000000000007F
:10018000000000000000000000000000000000006F
:10019000000000000000000000000000000000005F
:1001A000000000000000000000000000000000004F
:1001B000000000000000000000000000000000003F
:1001C000000000000000000000000000000000002F
:1001D000000000000000000000000000000000001F
:1001E000000000000000000000000000000000000F
:1001F0007545AD3DC3C5FD36FFFFFFFF6587214354
:1002000000000FE11F00C0E31B1080E301F02FE1AD
:100210007CD19FE507D0CDE3171080E301F02FE1FB
:1002200070D19FE507D0CDE3121080E301F02FE1FC
:1002300064D19FE507D0CDE3111080E301F02FE1F9
:1002400058D19FE507D0CDE3131080E301F02FE1F3
:100250004CD19FE507D0CDE31F1080E301F02FE1E3
:1002600040D19FE507D0CDE33C019FE53C119FE5E0
:100270003C219FE52E0000EB38019FE538119FE5FA
:1002800038219FE52A0000EB34019FE534119FE5FA
:1002900034219FE5260000EB30019FE530119FE5FA
:1002A00030219FE5220000EB2C019FE52C119FE5FA
:1002B0002C219FE51E0000EB28019FE528119FE5FA
:1002C00028219FE51A0000EB24019FE524119FE5FA
:1002D0000020A0E3280000EB1C019FE51C119FE516
:1002E000001041E0080051E30020A0A3042080A4F6
:1002F000001080A5D8009FE5D8109FE5010050E1CF
:100300000500000A042090E403002DE90FE0A0E1BD
:1003100012FF2FE10300BDE8F7FFFFEA0000A0E3B2
:100320000010A0E3D8209FE50FE0A0E112FF2FE12D
:10033000FEFFFFEA010050E10EF0A001012052E0B3
:100340000EF0A001013080E1023083E1030013E3ED
:100350000400001A043090E4043081E4042052E2E6
:10036000FBFFFF1A0EF0A0E10130D0E40130C1E440
:10037000012052E2FBFFFF1A0EF0A0E1010050E164
:100380000EF0A0010120C0E4FBFFFFEA0000E0E363
:100390001EFF2FE1742700407427004074260040A0
:1003A000742700407427004074250040383F000047
:1003B0003C0000403C00004018050000180500000B
:1003C000A8350000383F00003C0000403C000040E1
:1003D000A8350000A8350000A8350000A8350000A9
:1003E000A8350000A8350000A8350000A835000099
:1003F000383F00003C000040741D0040741D004068
:1004000074210040D52300000000A0E10000A0E11D
:10041000FC009FE5881090E5020411E30500000A46
:100420000110A0E3801080E5AA10A0E38C1080E505
:100430005510A0E38C1080E50010A0E3801080E54B
:10044000AA10A0E38C1080E55510A0E38C1080E585
:10045000A01190E5201081E3A01180E5A01190E5A6
:10046000400011E3FCFFFF0A0110A0E30C1180E53E
:100470000B10A0E3841080E5AA10A0E38C1080E5A7
:100480005510A0E38C1080E50110A0E3801080E5FA
:10049000AA10A0E38C1080E55510A0E38C1080E535
:1004A0000310A0E3041180E50510A0E3081180E526
:1004B000881090E5010311E3FCFFFF0A0310A0E39D
:1004C000801080E5AA10A0E38C1080E55510A0E311
:1004D0008C1080E5881090E5020411E3FCFFFF0A10
:1004E0000010A0E3001080E50410A0E3041080E5F4
:1004F0000210A0E3001080E540FFFFEAFEFFFFEAE4
:10050000FEFFFFEAFEFFFFEAFEFFFFEAFEFFFFEA53
:080510001A0000EA00C01FE020
:1005180030B5039A002A04D00F4D8400641924686A
:100528001460002B0CD00D4A012514688540AC439B
:1005380014600B4C8000084D02191160401906E048
:100548000749800042180F211160034A8018036090
:10055800012030BC02BC084700F1FFFF0CF0FFFF90
:1005680000F2FFFF01231A1C8240101C014A106090
:10057800181C704710F0FFFF01002DE900004FE143
:10058800800010E30100BDE804F05E121F502DE961
:1005980020009FE5001F90E5000090E50FE0A0E136
:1005A80011FF2FE10030A0E308209FE5003F82E51E
:1005B8001F50BDE804F05EE200F0FFFF00B5124BEB
:1005C8001A680E231340042B01D00C2B16D10F4BA5
:1005D8000F491A8808780F49885401321204120CFE
:1005E8001A800D4A1988914201D900221A800B4AB3
:1005F800138801331B041B0C138003E0062B01D165
:10060800074B1B7801BC004708C000E03E080040CB
:1006180000C000E03E000040FF0700004008004026
:1006280014C000E010B5124B1A68C0218A43E121BA
:100638001A6009030A22884204D11A6840210A4331
:100648001A6004220B4B802118780B4C1970110684
:10065800090E2170094C002121701870084B042ADA
:1006680002D192221A6000E0196010BC01BC004758
:10067800A8C11FE00CC000E000C000E004C000E01A
:1006880028C000E013B5154B00241C80144B1C80B7
:10069800144B1C80144B1A6808210A431A60134B28
:1006A80003221A70124B87221A70124B0522E1207E
:1006B8001A604002FFF7B6FF0F4B50221A60012163
:1006C800221C0E4B06200094FFF722FF0620FFF79E
:1006D80049FF02F055FF13BC01BC00473E0800402B
:1006E8003C00004040080040C4C01FE00CC000E0CF
:1006F80008C000E004C000E000C002E0C50500003A
:10070800074B1A6805218A431A60064B1A680821A4
:100718008A431A60044B1A68C0218A431A607047DA
:1007280004C000E0C4C01FE0A8C11FE000B5044A2F
:10073800202311781942FCD0024B187001BC0047E5
:1007480014C000E000C000E0014B18887047C046A4
:100758004008004010B5104B1A88002AFCD00F4BF7
:100768000F491A888C5C01321204120C1A800D4A47
:100778001988914201D900221A8002F009FF064A1D
:100788001388013B1B041B0C138002F0F9FE201C8C
:1007980010BC02BC0847C046400800403C0000406E
:1007A8003E000040FF07000001207047012070470D
:1007B80001207047012070470120704701207047D1
:1007C800012070470120704701207047F0B5131CC5
:1007D8000E4E10E04488071901340D782404240CC7
:1007E800BD71448044880131B44201D90027478053
:1007F800013B1B041B0C002BECD18388D21812047C
:10080800120C8280F0BC01BC0047C046FF07000004
:10081800F0B5131C0E4E00250FE0048807190134AB
:10082800BF792404240C0F70048004880131B44279
:1008380000D90580013B1B041B0C002BEDD18388DC
:100848009A1A1204120C8280F0BC01BC0047C04600
:10085800FF07000038B50E4883884024A34202D819
:1008680084882406240E0B4D221C291CFFF7D0FF78
:10087800094B002C02D101221A7006E000221A70DE
:100888008220291C221C00F0CDFF38BC01BC004787
:100898008A100040481000408910004038B50D4CBF
:1008A800A188F8220C4BD20091420DDC0B4D00229E
:1008B8001A70291C022000F059FF0204120C201C97
:1008C800291CFFF783FF01E001221A7038BC01BC24
:1008D8000047C046420800408810004048100040C9
:1008E80008B500F07BFD08BC01BC004708B500F066
:1008F80057FC08BC01BC004713B56B46D8710C4CBB
:100908000C4BA2889A42FCD802F042FE6946201C91
:1009180007310122FFF75AFF02F032FE064B1B781F
:10092800002B01D0FFF796FF13BC01BC0047C0465F
:100938008A100040FF07000089100040014B98888A
:100948007047C0464208004013B56C46073402F0B1
:100958001FFE0548211C0122FFF75AFF02F010FE76
:10096800207816BC02BC084742080040074A00230A
:100978001380074A1370074A07491370074A116022
:10098800074A1360074A13607047C046941800402E
:10099800C41800409C18004001000100981800404D
:1009A80090180040A018004008B50020024900F047
:1009B800DDFE08BC01BC0047A418004010B5094C76
:1009C800A3880822934200D81A1C2168802000F0CE
:1009D80029FF23681B182360A388181AA08010BC5D
:1009E80001BC0047B818004010B5074C002021682A
:1009F80000F0BCFE23681B182360A388181AA08087
:100A080010BC01BC0047C046B818004008B500211A
:100A180080200A1C00F006FF08BC01BC004700004B
:100A280008B50020024900F0A1FE08BC01BC00473F
:100A3800AD18004000B5234A1378DB06DB0E012B06
:100A480008D0022B17D00020002B39D11E4A1F4B8B
:100A58001A6034E01E490878002831D011791D4AFF
:100A68001278002091422BD21B4A184910705070FE
:100A78000A60181C24E012798F2313408022134245
:100A880006D00F2280211A40490291400A1C01E039
:100A980001229A400E490878002801D119070FD180
:100AA8000E4B186810400BD00D4909680A4B0A40D4
:100AB800511E8A411A7000225A70044A136001209C
:100AC80002BC0847A418004094180040B818004019
:100AD8009C180040AC180040AD1800409818004021
:100AE8009018004070B52F4B1C78E406021CE40EE9
:100AF80002D0022C50D118E0DE78997836020E43E5
:100B0800012E4AD1284D002806D0301C00F02AFCBE
:100B18002B880222134305E0201C00F023FC2B88BD
:100B2800022293432B80341C37E018798F23184016
:100B38008023184205D00F2505405B02AB401D1CE1
:100B480001E001258540194B1C78002C25D00F2485
:100B5800044022D0164B1C682C401ED0114B9978AB
:100B6800DB7800241B020B43A34216D1A24207D014
:100B780000F0A6FD0F4B1A6815431D6001240CE018
:100B88000D4B1B6801242B4207D100F0C5FD094B12
:100B98001A68AA431A6000E00024201C70BC02BC3A
:100BA8000847C046A4180040941800409C1800400C
:100BB8009818004090180040A018004000B5074B56
:100BC8001A780020D20606D19B78802252421A4316
:100BD800034B1A70012002BC0847C046A418004005
:100BE800C418004010B5214B1878C006C00E38D183
:100BF800DA78022A07D0032A02D0012A32D105E086
:100C080099781B4A1FE099781A4B0CE01A4B1B4A3B
:100C18001A6012231EE0002A04D0DA789C781202A7
:100C280022439B1801301A788842F4D1101E19D03B
:100C3800114A13609A78DB781B0213430AE0002BF1
:100C480000D0D218013013788842F8D1181E09D084
:100C580009490A60084A91880120994202D993807B
:100C680000E0002010BC02BC0847C046A4180040A1
:100C7800EC350000A8350000B818004054360000D4
:100C880000B5054B1B780020DB0603D1034A044B53
:100C98001A60012002BC0847A41800409C180040B4
:100CA800B8180040F8B5564B1F78FF06FF0E002015
:100CB800002F00D0A0E09B78002B6DD171E0637805
:100CC800042B47D0052B47D0022B62D14C4B6279BD
:100CD8009B78934239D14B4A13704B4B22791A7047
:100CE8004A4B00221A705A709A70DA70484E0125E1
:100CF80001233268AB401A4202D0281C00F08AFC5B
:100D080080235B023268AB401A4203D0802028431C
:100D180000F080FC0135102DEAD13D4B3D4A1A60A8
:100D28003D4A002313603D4A0120136000F0E8FBB0
:100D3800E17901223A4B480602D519880A4302E0B4
:100D4800198891430A1C1A8023E0E378A2781B02D1
:100D580013431FE0E7781CE0002F1AD1A5788F23F2
:100D68001D408020054205D00F222A4043029340AF
:100D78001A1C01E00122AA40254B19680A431A608F
:100D8800201C00F0EFFB281C00F01AFC281C00F0C7
:100D98006DFC2378E41800E0224C2378002B8ED1D8
:100DA80023E0184A01241370194D261C331C2A68A5
:100DB800A3401A4202D0201C00F02CFC80235B02C6
:100DC8002A68A3401A4203D08020204300F022FC66
:100DD8000134102CEAD10E4B0E4A1A600E4B00203B
:100DE80018600E4B186000F08BFB064B1878044B0C
:100DF8009B78C01A43425841F8BC02BC0847C04619
:100E0800A41800409C180040AC180040C0180040CE
:100E1800981800400100010090180040A0180040F8
:100E280094180040A835000000B50C4A1378DB067A
:100E3800DB0E0020012B0ED10949087800280AD0C2
:100E48000849127909780020914204D906498A187C
:100E580006490A60181C02BC0847C046A41800408E
:100E68009C180040AC180040C0180040B81800405A
:100E7800F0B5434B1A78D20685B0D20E0025012A68
:100E880078D1404A1578002D74D000250395029535
:100E98002E1C01953C4C6AE06378042B0DD0052B81
:100EA80021D0022B61D1374B62791B789A425CD0F2
:100EB800E378A2781B02134358E0A2780192304AE3
:100EC80013790022E6780392019A9A424DD12C4A6E
:100ED80093789E4249D12D4B019A9A5C0292019ACD
:100EE80001259E5441E0264B019A1B799A423CD138
:100EF800A2788F231A40802300921A4205D00F2728
:100F080017405B02BB401F1C02E0009B01279F406B
:100F18001B4B9B789E4214D11D4B1A683A431A60AA
:100F28001C4B1A68BA431A60201C00F01BFB00987F
:100F380000F046FB009800F099FB039A3A430392AD
:100F480013E0029B9E4210D1039A02963A420CD1BA
:100F58000F4B1A68FF433A401A600E4B1A68174045
:100F68001F60009800F056FB02962378E418237857
:100F7800002B91D105B0281CF0BC02BC0847C04624
:100F8800A41800409C180040A8350000C018004074
:100F9800981800409018004070B5041C012000F01B
:100FA80059FE601E062800D9EFE001F06DFC04A48C
:100FB800D8EEEEE9EB00FFF7F7FC754D2878C0098D
:100FC80000F0FCFAEB79AA79724C1B021343A38058
:100FD8002B785A06920F03D0012A00D084E034E01F
:100FE80068780B2800D97FE001F04EFC06097E0BDB
:100FF8007E0F12151B1E272CFFF71CFD1FE000207B
:1010080000E00120FFF76EFDA1E0FFF7D7FD9EE0AD
:10101800FFF7E8FD13E0002000F052FB0023A38057
:10102800B3E0FFF72DFE0AE0FFF73CFE00285BD097
:10103800FFF7ECFC00F05EFCA7E0FFF7F5FE0028E8
:1010480052D091E0FFF714FF81E0DB06DB0E012BA5
:101058004AD12B79012B47D86B78042B24D008D898
:10106800012B11D0002B26D0022B24D0032B3BD1EF
:101078000DE0212B22D002D8202B35D11BE0222BCA
:1010880023D0232B30D127E0FFF790FB18E0404B0B
:10109800D8789A7800021043FFF78CFB002823D0F9
:1010A8003D4A3C4B1A605FE0E878AB780002184391
:1010B800FFF782FB4BE0384B236066E0FFF780FBCD
:1010C800002811D0344B23604EE0E878AB7800025A
:1010D8001843FFF777FB3AE02D4BD8789A7800024F
:1010E8001043FFF771FB32E0802000F0E9FA294B4A
:1010F80000229A8049E0264D2B78DB092CD1254C1B
:10110800A388002B41D0FFF76FFCA388002B3CD1AC
:101118002B785A06920F012AE6D1DB06DB0E012B4B
:10112800E2D12B79012BDFD86B78022B06D0202B4C
:101138000BD0002BD8D1FFF737FB08E0E878AB7865
:1011480000021843FFF734FB01E0FFF737FB0028E4
:10115800CAD0FFF75BFC18E0FFF762FC15E00C4B08
:101168001B787F22934302D0FFF728FC0DE00B4B3E
:101178001878010609D51040187000F0F5F804E059
:10118800002000E0802000F0C7FA70BC01BC0047D6
:10119800A4180040B8180040AD180040C41800401A
:1011A80000B503048020400018430B4B10221A603E
:1011B8000A4A0B4B0B491A6010220B681A42FCD0E2
:1011C800054B10221A60064B064918600B681A4234
:1011D800FCD001BC0047C04608C2E0FF0005FE0085
:1011E80010C2E0FF00C2E0FF00B50E4900230B600B
:1011F8000D4B082201201A6008601A600B498022F2
:1012080052000B681342FCD0094A01235B42136069
:10121800084A1360084A1360084B0C221A6001BC84
:101228000047C04648C2E0FF4CC2E0FF00C2E0FFF2
:1012380038C2E0FF34C2E0FF08C2E0FF04C2E0FFAA
:10124800F8B54F464646C0B43B493C4B08683C4A53
:10125800186081461060000720D530221A60394A8C
:10126800394B1A6010220B681A42FCD0334B3022DB
:101278001A60364A344B30491A6020220B681A42E9
:10128800FCD0334B1B68DA0650D42C4B4846186008
:101298000CBC90469946F8BC01BC00474B465B071E
:1012A800F3D52C4E01273368002BEED000242A48B2
:1012B8003B1C3268A340012580461A421DD0424695
:1012C8001D491360600820220B681A42FCD0204B8D
:1012D8001B68274214D1002C1DD15A071BD51F4A61
:1012E8001368002B18D0012000F03AF801343B1C99
:1012F8003268A34001351A42E1D1202DF6D1D2E758
:10130800164A80001358002BF7D0032000F028F865
:10131800202DEBD1C7E7114A80001358002BECD0E1
:10132800022000F01DF8202DE0D1BCE7FFF75CFF9C
:1013380000F0D9FAA9E7C04600C2E0FF08C2E0FF02
:10134800C81800400005FE0010C2E0FF0002FE00C1
:1013580014C2E0FF30C2E0FF38C2E0FF6836000088
:101368001847C0467047C04600B580231843030499
:10137800802040001843154B10221A60144A154B60
:1013880015491A6010220B681A42FCD00F4B102224
:101398001A60104B104918600B681A42FCD00B4BAE
:1013A80010221A600A4A0B4B0B491A6010220B686C
:1013B8001A42FCD0054B10221A60064B06491860E9
:1013C8000B681A42FCD001BC0047C04608C2E0FFC7
:1013D8000005D00010C2E0FF00C2E0FF10B53A4B94
:1013E8008022196812060A43384C1A601A232360AF
:1013F80082B000F053FB364B984226D000F04EFBEB
:10140800344B984221D01F23236033491F220B6895
:1014180013401F2BFBD1314B314A19680A401A601F
:101428008022196892050A431A602E4B1A689200A6
:1014380092081A6080221968D2050A431A602A4B5A
:10144800196803220A431A6024E0204B12221A600A
:1014580021490B681340122BFBD1244B244A1968ED
:101468000A401A6080221968D2020A431A601D4B8A
:10147800204A19680A401A6080221968D2040A436F
:101488001A60174A19680A401A60802219685205BA
:101498000A431A6000230221002200931620164BEB
:1014A800FFF736F81620FFF75DF802F069F8FFF746
:1014B8009BFE0020FFF758FF104B092202B01A606C
:1014C80010BC01BC0047C046C4C01FE0F4CFE0FF19
:1014D80035FF001735F90018F8CFE0FF00C002E02B
:1014E800FFFFFFCF04C002E010C1E0FF10C002E020
:1014F800FFFFF3FFFFFFFFF34912000004C2E0FF04
:1015080000B50304802040001843114B10221A60D4
:10151800104A114B11491A6010220B681A42FCD06C
:101528000B4B10221A600C4B0C4918600B681A42BE
:10153800FCD00B4B03221A600849802252000B682A
:101548001342FCD0024B802252001A6001BC0047B3
:1015580008C2E0FF0005D80010C2E0FF00C2E0FFAB
:1015680044C2E0FF10B582780F2313405B00D20914
:101578009B180D4A012114689940214311600B4AB8
:1015880013604279037912021A43094B09491A6018
:10159800802252000B681342FCD0074B8022520075
:1015A8001A6010BC01BC004744C2E0FF48C2E0FF1B
:1015B8004CC2E0FF00C2E0FF08C2E0FF7047C0462F
:1015C80000B50F23034000065B00C00F0D4A1B182F
:1015D8001B0413430C4A102111600C4A0C49136078
:1015E80010220B681A42FCD0074B10221A60802286
:1015F800064B520006491A6010220B681A42FCD0AA
:1016080001BC00470005400008C2E0FF10C2E0FF2F
:1016180000C2E0FF00B50F23034000065B00C00FC7
:101628000D4A1B181B0413430C4A102111600C4A65
:101638000C49136010220B681A42FCD0074B102289
:101648001A60094A064B07491A6010220B681A42A9
:10165800FCD001BC0047C0460005400008C2E0FFBE
:1016680010C2E0FF00C2E0FF0001200000B50F2318
:10167800034000065B00C00F0D4A1B181B041343F0
:101688000C4A102111600C4A0C49136010220B6897
:101698001A42FCD0074B10221A608022064B5200D7
:1016A80006491A6010220B681A42FCD001BC004798
:1016B8000005400008C2E0FF10C2E0FF00C2E0FFE2
:1016C80000B50F23034000065B00C00F0D4A1B182E
:1016D8001B0413430C4A102111600C4A0C49136077
:1016E80010220B681A42FCD0074B10221A60094AD4
:1016F800064B07491A6010220B681A42FCD001BC3D
:101708000047C0460005400008C2E0FF10C2E0FFE5
:1017180000C2E0FF0001010000B50F2303400006EE
:101728005B00C00F0D4A1B181B0413430C4A102101
:1017380011600C4A0C49136010220B681A42FCD045
:10174800074B10221A608022064B520006491A6085
:1017580010220B681A42FCD001BC0047000540006B
:1017680008C2E0FF10C2E0FF00C2E0FFF0B50F22A0
:101778000240031C9446900001221043214A224C47
:1017880010608022120120681042FCD08005800D74
:10179800C61CB6080DD01D4F00243A68150A0A70F9
:1017A8004D700134150C120E8D70CA700431B4429C
:1017B800F3D1144A00211160154A1A41D1071DD4EA
:1017C80061461B064A00DB0FD218A023DB00120477
:1017D8001A43104B302119600F4B10491A60102220
:1017E8000B681A42FCD00B4B30221A600C4A0A4B89
:1017F8000A491A6010220B681A42FCD0F0BC02BCDD
:101808000847C04628C2E0FF20C2E0FF18C2E0FF38
:101818004812000008C2E0FF10C2E0FF00C2E0FF6B
:101828000005F200F0B50F2303409C009C460223FC
:101838001C431E4B1C601E4BD61C1A60B60810D0E9
:101848001C4F0023CC788D7824022C434D78240239
:101858002C430D7824022C4301333C600431B342FD
:10186800F0D1124B00211960000661464B00C00FF1
:101878001B18A021C9001B040B430F493020086026
:101888000E490F480B60102103681942FCD00A4B1F
:10189800302119600B49094B094819601021036868
:1018A8001942FCD0101CF0BC02BC084728C2E0FF5B
:1018B80024C2E0FF1CC2E0FF08C2E0FF10C2E0FF44
:1018C80000C2E0FF0005FA00704708B5022802D000
:1018D800032805D102E0FEF7E1FF01E0FEF7BAFFB9
:1018E80008BC01BC004708B5FFF740F808BC01BCBC
:1018F8000047000008B5044B1B78002B01D0FEF709
:10190800A9FF08BC01BC00479C1800407FB53223E2
:1019180001930290039101F03BFE01A804A9044B36
:1019280000F008F801F02CFE049807B002BC084744
:10193800F1FFFF7F1847C046F0B51D4A0E1C411E37
:101948008BB089190432002300E02B1C10CA5D1CDF
:10195800A04203D21D1C1B24154B02E01B2DF4D101
:10196800F9E7A200D258914202D8013C002CF8D1E4
:10197800281C211CFFF7CAFF0027B84212D13423C4
:1019880001930C4B02950493039401F001FE0A4B5A
:1019980001A806A900F012F801F0F2FD069BBB426F
:1019A80000D1371C0BB0381CF0BC02BC0847C0463D
:1019B800A836000040190100F1FFFF7F1847C04614
:1019C800F0B58FB0071C002002928B05834249D1E5
:1019D8008E0AB202D319351C3C1C019203933EE0D7
:1019E800039A9446012252429444204A0023043226
:1019F80000E0031C02CA581C8C4203D2181C1B218D
:101A08001A4B02E01B28F4D1F9E78A00D258944512
:101A180002D801390029F8D1FFF778FF002817D13B
:101A2800029A33230593D31B1B1907938023DB00EA
:101A380008930F4B0694099301F0AAFD0D4B05A8D6
:101A48000AA900F019F801F09BFD0A9B002B02D0AF
:101A5800751BA80206E08023DB00013DE418002D79
:101A6800BED101980FB0F0BC02BC0847A8360000F0
:101A780040190100F1FFFF7F1847C04610B5131E3B
:101A880008D00B18121A02E00488845202309842D7
:101A9800FAD30B1C181C10BC02BC08471FB5362310
:101AA800039301F075FD03A801A9044B00F008F8A1
:101AB80001F066FD029805B002BC0847F1FFFF7F00
:101AC8001847C04600B540000B09002A02D0012A79
:101AD8001BD10EE05A1E9341C018174BC018800046
:101AE8001F2249000368114003228A409343036080
:101AF8001FE05A1E9341C0180F4BC0181F228000C8
:101B080049001140036803220FE05A1E9341C01890
:101B1800094BC01880001F224900036811400122A8
:101B28008A4093430360036802228A40111C1943C8
:101B3800016001BC0047C04610B0003870B50B0901
:101B480044005D1EAB41E318114C1B199B004E006D
:101B58001F251C6835400326AE40B4431C60002A8C
:101B68000AD0012A10D10B4BC018400103688A40E3
:101B7800111C1943016007E0064C00194001036875
:101B880001228A409343036070BC01BC0047C046F1
:101B980000B0003800FEFF01054B4001C018006886
:101BA80001238B401840C11A484248417047C0463B
:101BB80014C0FF3F8020C0017047000007B5002314
:101BC8000093094A0AE0019302E001990131019169
:101BD80001999142F9DD0099013100910099814202
:101BE800F1D303B001BC0047040D000038B50B4C1D
:101BF8000121201C00F087F80220FFF7DFFF201CDE
:101C080000F0A5F8051C201C00F090F801204540C4
:101C18002806000E38BC02BC0847C0460302000074
:101C280038B50B4C0121201C00F06DF80220FFF79D
:101C3800C5FF201C00F08BF8051C201C00F076F86E
:101C4800012045402806000E38BC02BC0847C046A3
:101C58000A02000008B5FFF7B1FF08BC01BC004745
:101C6800704708B5FC210020C90200F046F808BCFE
:101C780001BC004708B58020F421C001C90200F06A
:101C88003CF808BC01BC004737B580246D46E40128
:101C980006352A1C201C022100F029F82A88074B47
:101CA8009A4206D1FC230234DB029C42F1D1012086
:101CB80000E000203EBC02BC0847C046FFFF000011
:101CC80008B58823DB0100F003F808BC01BC004715
:101CD80018470120704770477047704708B5FFF7ED
:101CE8006FFEC317181AC00F08BC02BC084708B516
:101CF800FFF7C4FE08BC01BC004708B5FFF71CFE8F
:101D080008BC01BC004770B50406050A240E0E1C69
:101D1800281C211C0022FFF711FF0122B243281CB6
:101D2800211CFFF7CFFE70BC01BC004738B5040684
:101D3800050A240E281C211C0022FFF7FFFE281C80
:101D4800211C0022FFF7BEFE38BC01BC004708B5C5
:101D5800011C0906000A090EFFF71EFF431E9841E1
:101D680008BC02BC084708B5FEF78CFC08BC01BCDF
:101D7800004708B5FEF7C4FC08BC01BC004708B51D
:101D8800FEF750FC08BC01BC004708B5FEF7DCFCB8
:101D9800C317181AC00F08BC02BC084708B5FEF7DD
:101DA800C5FC08BC01BC004708B5FEF7D3FC08BC5D
:101DB80002BC084708B5FEF793FD0120FEF796FD23
:101DC800024B01221A7008BC01BC0047CC18004025
:101DD80010B5064C2378002B04D00020FEF786FDB2
:101DE8000023237010BC01BC0047C046CC1800403B
:101DF800704708B5FEF7A2FDC317181AC00F08BC34
:101E080002BC084708B5FEF777FD08BC01BC0047CF
:101E180008B5FFF7EEFF0028FBD0FEF795FD08BCDC
:101E280002BC084708B50B4800F0B4FB00F0B8FB4B
:101E38000378792B01D0592B06D14378002B03D195
:101E4800012008BC02BC0847034800F0A3FB00209F
:101E5800F7E7C046183700002C37000010B5054CCE
:101E68002378002B02D1044800F094FB207810BCA2
:101E780002BC0847CD1800403637000008B50448B2
:101E880000F088FB034800F085FB08BC01BC004754
:101E9800473700004E37000008B5044800F07AFBC9
:101EA800034800F077FB08BC01BC0047523700002C
:101EB8004E37000008B5FFF7B5FF00280CD0084BD7
:101EC800E1201B68000300F00FF8FA204000FFF73C
:101ED80075FE044800F05EFB08BC01BC0047C04624
:101EE8005C1900404E3700001847C046F0B585B071
:101EF8000190FFF797FF00285DD0314800F04AFBBA
:101F0800FFF7EBFE00F064FB00F0A4FB041E41D0D9
:101F1800019B002B04D08021201CC90000F028FC64
:101F2800A38922680293274B6568A7689A4238D12B
:101F3800281C391CFFF7E1FE00F084FBEB192C1C70
:101F4800039316E000F086FB061E23D0019B002BAE
:101F580004D08021301CC90000F00AFC8021201C1C
:101F6800C900321CFFF7BAFE00F06CFB8023DB00CF
:101F7800E418039B9C42E5D300F04CFB281C391C59
:101F880000F03CFA029B83420BD10F4800F002FBA1
:101F98000E480CE000F049FB0B4800F0FBFA0C4837
:101FA80005E000F042FB084800F0F4FA094800F0A8
:101FB800F1FAFFF791FE05B0F0BC01BC0047C0463E
:101FC80059370000C3C5FD36DC3A00004E37000023
:101FD8006437000090370000F0B5C3B0FFF73EFF4C
:101FE800002800D193E04C4800F0D4FA00F0A8FA99
:101FF800061C00F0A5FA041C00F0A2FA2402000452
:10200800044300F09DFA050600F09AFA3443061CD2
:1020180000F096FA2543041C00F092FA240200040A
:10202800044300F08DFA344300060443211C281CA5
:1020380000F0E4F900902806000EFF2600F06AFA86
:102048003602281C3040000AFF2700F063FA3F04DC
:10205800281C3840000C00F05DFA280E00F05AFAEF
:102068002006000E264000F055FA2740300A00F0FE
:1020780051FA380C00F04EFA200E00F04BFA009A94
:102088001006000E00F046FA009B180A0006000E23
:1020980000F040FA2606220A0192360E171C009517
:1020A80019E080210098490002AAFFF720FE0024C9
:1020B80008231B196A46985C00F02CFA002C01D101
:1020C800FFF709FE802301345B009C42F0D1009A9F
:1020D800D2180092013F002FE3D1019B180240194A
:1020E800002E11D0311C02AAFFF701FE3C1C082269
:1020F80012196B46D05C00F00DFA002C01D1FFF7E5
:10210800EAFD0134B442F2D1044800F043FA43B086
:10211800F0BC01BC0047C046593700004E370000EC
:1021280008B5FFF77FFE002807D0054800F032FA0F
:10213800FFF7A0FD034800F02DFA08BC01BC0047DA
:10214800AE3700004E37000008B5FFF787FE0028BD
:102158000ED0FFF799FD4E23002800D05923181CF4
:1021680000F0D8F9044800F015FA044800F012FA13
:1021780008BC01BC0047C046DC3A00004E370000EE
:1021880008B5FFF74FFE002812D000F075F80028B8
:1021980001D1094804E000F057F8002803D10748A6
:1021A80000F0F8F904E0064800F0F4F900F090F8BF
:1021B80008BC01BC0047C046B9370000E43700003E
:1021C8000438000008B5FFF749FE00280BD0FFF7D8
:1021D80029FE002807D0054800F0DCF9FFF741FD8B
:1021E800034800F0D7F908BC01BC0047AE3700002F
:1021F8004E37000010B5104800F0CCF900F0D0F9C7
:10220800021C1378111A0132002BFAD1C843101896
:102218000A290ED1094AC45CD15C8C4209D1013328
:102228000A2BF8D1064800F0B5F9064B01221A70BE
:10223800002010BC02BC08473637000010380000E8
:102248004E370000CD18004038B5FFF7B3FC031C2B
:102258001D68084A99689C8940680023954204D102
:1022680000F0CCF8241A63426341181C38BC02BC45
:102278000847C0467545AD3D08B5FFF79BFC0268A9
:1022880083890020013203D0034A9818431E9841DD
:1022980008BC02BC0847C0460100FFFF08B50A4B4E
:1022A8000A4A1968914203D100221A60012007E006
:1022B800FFF7CAFF031C0120002B01D0FFF7B0FC79
:1022C80008BC02BC0847C046F8FF004038023DC6BB
:1022D80008B500F00DF9044A044B1A60FFF7F0FC4A
:1022E800034800F057F9FEE78393A484FCFF0040FD
:1022F8001B38000010B5304C01E000F021F92368CC
:1023080000F062F80028F8D12C4800F043F92C4876
:1023180000F040F92B4C00F043F94378002B01D032
:10232800284822E00078413837281DD800F0ACFA58
:102338003E32383B2C1C1C1C351C1C1C1C231C1C32
:102348001C2F1C1C28201C261C1C1C1C1C1C1C1C98
:102358003E32383B2C1C1C1C351C1C1C1C231C1C12
:102368001C2F1C1C28201C26201C00F013F9D2E767
:10237800FFF784FDCFE7FFF78FFDCCE7012000E0F2
:102388000020FFF7B3FDC6E7FFF7CAFEC3E7FFF774
:10239800F7FEC0E7FFF78EFDBDE7FFF7D5FEBAE70A
:1023A800FFF710FFB7E7FFF717FEB4E7FFF722FFC5
:1023B8000028B2D1AFE7C046D01800405C38000012
:1023C8004E370000363700001847C04610B5FFF7F3
:1023D80080FC041CFFF744FC00F028F8002C07D010
:1023E800FFF75CFF002801D0FFF784FFFFF770FFBD
:1023F800014800F0CFF8FEE79D38000070B50022D4
:10240800031C094C101C09E09E5C051275406D0008
:102418002D5B000268400004000C01328A42F3DBA5
:1024280070BC02BC0847C046DA38000010B5144B2F
:1024380000221A70FFF7DAFB124C1349134A144BA7
:1024480000280CD013482060134808601349116015
:10245800134A1A60134A144B1A60144A0BE01448C2
:1024680020601448086014491160144A1A60144A1C
:102478000D4B1A60134A144B1A6010BC01BC00477C
:102488006419004060190040681900405C19004058
:10249800D01800406F1D00007B1D0000871D000044
:1024A800931D0000A51D000054190040B11D000037
:1024B800BD1D0000D91D0000F91D0000FB1D000016
:1024C8000D1E0000191E00005819004008B5054BE4
:1024D8001B6800F00BF8044B01221A7008BC01BC01
:1024E8000047C04660190040641900401847C046BC
:1024F80008B5054B1B6800F00BF8044B00221A7056
:1025080008BC01BC0047C046681900406419004077
:102518001847C04610B5074B1B78041C002B01D187
:10252800FFF7D4FF044B201C1B6800F007F810BC11
:1025380001BC004764190040541900401847C046C0
:1025480008B5064B1B78002B01D1FFF7BFFF044BE2
:102558001B6800F007F808BC02BC08476419004073
:10256800581900401847C04610B5041C02E0013451
:10257800FFF7D0FF20780028F9D1054C02E001349C
:10258800FFF7C8FF20780028F9D110BC01BC00472C
:10259800DA3A000008B5FFF7E7FF08BC01BC0047BE
:1025A80070B50A4D00247F26FFF7CAFF031C285583
:1025B800281C0A2B04D00D2B02D001343440F3E739
:1025C8000023035570BC02BC0847C046D41800401D
:1025D80038B500250B4C09E0281C0B4900F0D4FF46
:1025E8000135002902D14320FFF794FF236800F04A
:1025F8000FF80028F0D0054B01221A7038BC01BC36
:102608000047C046D0180040102700006C1D00404D
:102618001847C04608B5FFF793FF0428FBD10620EA
:10262800FFF778FF08BC01BC004708B51520FFF785
:1026380071FF1820FFF76EFF1820FFF76BFF08BC2B
:1026480001BC004708B50620FFF764FF08BC01BCC1
:102658000047000070B5FFF773FF041CFFF770FF19
:10266800013C2406051C240EFFF76AFF012C27D81D
:1026780028430006000EFF2822D1144B1B78AB42DA
:102688001ED18024124E0025E400FFF759FFA855FB
:102698000135A542F9D1FFF753FF0406FFF750FFB4
:1026A800240C04432404301C291C240CFFF7A6FE28
:1026B800844205D1054B1A7801321A70301C02E0A9
:1026C800FFF7B3FF002070BC02BC08476C1D004038
:1026D8006C190040F7B54278837812021B041A433C
:1026E80003781A43C3781B061A4341798379090290
:1026F8001B040B4301790B43C17909060B43194DA0
:1027080019490324CE0A2640B6007759CF190097F5
:10271800560917017740BE18009F7E409B1B134E39
:1027280089190E1C2640B6007759CF1900971E014B
:102738005F097E40009FF6187E40921B0029E1D178
:10274800110A02704170110C120EC2701A0A03713C
:1027580042711A0C1B0E81708271C371F7BC01BCE7
:102768000047C046E03A00002037EFC64786C861F8
:1027780070B5051C0E1C002403E02819FFF7AAFFFA
:102788000834B442F9D370BC01BC00470000000013
:10279800000000000000000000000FE18000C0E31E
:1027A80000F021E11EFF2FE100000FE1800080E32F
:1027B80000F021E11EFF2FE1100E10EE010010E3E2
:1027C800FCFFFF0A100E11EE1EFF2FE10000A0E132
:1027D8000000A0E10000A0E102002DE9101E10EEAB
:1027E800020011E3FCFFFF1A100E01EE0200BDE823
:1027F8001EFF2FE10000A0E12047C0460847C04661
:102808001047C0461847C0460047C0462847C0463C
:102818006847C0463847C0464047C0464847C04654
:102828005047C0463047C0467047C0466047C0461C
:102838005847C04603B47146490840004900095E3C
:1028480049008E4403BC704703B4714602318908BD
:102858008000890008584018864603BCF746C046E1
:1028680002B4714649084900095649008E4402BC21
:102878007047C04603B47146490840004900095AE8
:1028880049008E4403BC704702B4714649084900A8
:10289800095C49008E4402BC7047C0460000000035
:1028A80000000000000000000020B0E32030B0E38A
:1028B800010052E1012042200000B0E00220A2E025
:1028C800013053E2F9FFFF1A010052E101204220D2
:1028D8000000B0E00210A0E11EFF2FE10000A0E11F
:1028E8000000A0E10000A0E1F0B55F4656464D4665
:1028F8004446F0B48BB080460C1C0592002303605C
:102908009B462EE2651C252906D0404600F0D0FCE7
:102918002C1C26E2251C09E05E4610218A4620224E
:10292800914680231B029C468027402128786C1CF6
:10293800031C203B1A06120E102A15D81B069B0DE5
:10294800C24AD3589F460E43E4E73E43E2E7634654
:102958001E43DFE748460643DCE752461643D9E7FD
:1029680080239B001E43D5E7321C2A2807D0021C6F
:10297800303A1206120E5B46092A0CD918E0059B5C
:10298800191D05911B68002B02DA5B4210261643BD
:102998006878AC1C0CE09A00D3185B0030381B1820
:1029A80020780134021C303A1206120E092AF2D994
:1029B8009A46DB43DB17514619408A46D9462E28EA
:1029C80027D120782A2807D00134031C303B1B0666
:1029D8001B0E092B08D919E0059B1A1D05921A68C8
:1029E8009146607802340EE05B469A00D3185B008B
:1029F80030381B1820780134021C303A1206120EA7
:102A0800092AF2D999464B46002B02DB80235B004A
:102A18001E4368280AD12078682804D108231E4359
:102A28006078023402E0013404231E43782803D876
:102A38008300874AD3589F46864B1D68002D00D1D6
:102A48008FE14946009105AB01934146321C53463C
:102A580000F0A3F985E14046252100F029FC80E13A
:102A6800059B1A1D05921D78012252429244301C82
:102A78005146424600F04EFC4046291C00F018FC26
:102A8800F30600D46DE120205146424600F032FCA6
:102A980067E1300707D5059B1A1D05921B6841465B
:102AA8000A681A705DE1059B1A1D05921B6840466D
:102AB80002681A6055E1059B1A1D05921D68281CBD
:102AC80000F07EFC071CF10506D50123814500DBDB
:102AD80000231B0600D04F465246D21B9246301C9C
:102AE800111C424600F016FC002FC9D0231C444696
:102AF800B0461E1C2978201C00F0DAFB0135013F86
:102B0800002FF7D1331C4646A0461C1CB8E7059B8E
:102B18001A1D05921D6833062321DB1719400391FE
:102B280080235B001E430822914659E080239B01C5
:102B38001E4359460391320606D5782802D1464BE2
:102B4800039301E045490391F20518D5444B1E4013
:102B580015E033063021DB1719400391F2050ED535
:102B68003F4B1E400BE059460391F20507D53C4BFD
:102B78001E4004E08023DB011E435B46039371047F
:102B880017D5059B1A1D05921D68720702D52D04DD
:102B98002D1403E0330701D52D062D0E002D03DA81
:102BA8006D422D21039117E0B20610D4730611D49B
:102BB80012E0059B1A1D05921D68710702D52D04A8
:102BC8002D0C09E0320707D52D062D0E04E02B2326
:102BD800039301E020210391F20503D5204B1E4009
:102BE800F30501D401218946583803061B0E202B12
:102BF80066D80006800D1B4B1B589F465F46072171
:102C0800002D35D15DE05F46002D3AD159E05F4691
:102C1800002D56D080239B013340134A94460F223F
:102C28000494002B06D0111C2940104C605C07A9A5
:102C3800785405E0111C29406446605C07A9785463
:102C480001372D09EDD1049C3BE0C046F03A000065
:102C5800343B0000701D0040783000005830000000
:102C6800FFFDFFFF183D0000EC3E0000FC3E0000A9
:102C78000A1C2A40303207ABFA540137ED08F7D165
:102C88001FE080231B02334004930498002807D0D8
:102C980003233B40032B03D107AB2C21D955013724
:102CA800281C0A2100F070FC303107ABD9550137D8
:102CB800281C0A2100F060FC051C0028E5D100E072
:102CC8005F464A46D51BEB43DB171D405046431B66
:102CD800DB1B9A46FF2303998B429B415B4252467A
:102CE800D21A92460B1C5A1E93415046C01A82466D
:102CF800802189000E4205D1301C5146424600F021
:102D080009FBDA46039AFF2A03D9110A404600F064
:102D1800CFFA039B002B04D01906090E404600F099
:102D2800C7FA301C5146424600F0F4FA3020291CFC
:102D3800424600F0DFFA7D1E0CD4371C261C4446A0
:102D480007ABE95C201C00F0B3FA013DF8D2A046BD
:102D5800341C3E1CF00604D520205146424600F0A3
:102D6800C9FA2178002900D0CCE541468B68002BB0
:102D780005D00A6849688A4201D20021995442461E
:102D8800106801E0012040420BB03CBC90469946D7
:102D9800A246AB46F0BC02BC0847284710B5041C45
:102DA8000B78002B05D0431C06D04B68013B4B60C9
:102DB80002E08B6800F004F8201C10BC02BC084735
:102DC8001847C046F0B55F4656464D464446F0B4EF
:102DD80083B082460191904699460C9F012676421F
:102DE80000E02E1C751C504600F04CFA041C00F044
:102DF800DBFA0028F5D1611C00D187E04D4B414634
:102E080019408846002F3BDD09060ED52B2C06D02D
:102E18002D2C0AD18023DB0042461A439046B51C6C
:102E2800504600F02FFA041C013F002F28DD302CFB
:102E380026D180239B00414619438846013F6E1CDA
:102E4800504600F01FFA041C002F15DD782801D029
:102E5800582811D14A46002A01D0102A0CD1364BE5
:102E6800414619408846013FAE1C504600F00AFA18
:102E7800041C102291465AE04B46002B55D056E0D0
:102E88004946002901D10A2291460026002F11DC6B
:102E980019E0434659460B439846013F321C4E46BB
:102EA800564386190135504600F0ECF9041C002FF2
:102EB80003D108E080239B009B46201C494600F074
:102EC8004FFA0028E5DA201C5146FFF767FF434612
:102ED8009B051ED54146C9071DD4019A13681A1DC2
:102EE80001990A601A689023DB004146194099420B
:102EF80000D176424346DB0601D516700BE0414609
:102F0800090701D5168006E0166004E001256D4228
:102F180001E002256D42281C03B03CBC904699464E
:102F2800A246AB46F0BC02BC084708229146351CB5
:102F3800ABE7C046FFF9FFFFFFFDFFFFF0B55F46B7
:102F480056464D464446F0B489B003900F1C07928C
:102F58000020814600210491C24A924620239B46C4
:102F680038787C1C002800D182E1252838D0061C3E
:102F780000F01AFA002801D11AE02C1C651C2078F0
:102F880000F012FA0028F8D1261C4C46039F00E0F6
:102F98000134381C00F076F9051C00F005FA002809
:102FA800F6D1A146281C0399FFF7F8FE371CD7E78E
:102FB800039800F067F9B04203D101208144271C2F
:102FC800CEE7051C0399FFF7E9FE013500D04FE174
:102FD8000499002900D04BE101235B42049347E1A7
:102FE8007B78002290462A2B02D1BC1C01239846EC
:102FF800002547460CE0554500DD39E1AB005D1979
:103008006D00303EAD1900D532E1584607434446BD
:103018002678611C8846301C00F09AF90028EAD10D
:103028004346B8461F1C331C42465846104200D13E
:103038008D4D4C2B05D16678A71C44231A43904626
:103048000EE0682B0CD16678682E05D110231A4340
:103058009046A678E71C03E0A71C08231A4390466D
:10306800253E532E00D903E1B600804B9B599F465D
:10307800039800F007F9252802D1012189446FE758
:10308800041C0399FFF78AFE013400D0F0E0049A8B
:10309800002A00D0ECE001235B420493E8E05B46A1
:1030A8004046034200D10125012441460C40002638
:1030B800002C03D1079B1A1D07921E68002D00D112
:1030C800D6E01ADDB846271C4C46039800F0DAF81B
:1030D800421C07D1049B002B00D0C9E001235B42AE
:1030E8000493C5E0002F01D1307001360134013D51
:1030F800002DEAD1A1463C1C47466342634104982F
:10310800C01804902CE7802241460A430095039892
:1031180007A90A23FFF756FE041C8DE080224346C8
:103128001A430095039807A90023FFF74BFE041CD8
:1031380082E04046C00700D512E7079B1A1D079298
:103148001B684146C90602D54A461A7008E7404638
:10315800000702D54946198002E74A461A60FFE689
:10316800802243461A430095039807A90823FFF7CE
:1031780029FE041C60E01E2342469A4300950398EA
:1031880007A91023FFF71EFE041C55E00124644222
:103198000134039800F076F8061C00F005F90028C1
:1031A800F6D1701C30D00123414619400691002207
:1031B8000592002904D1079B1A1D07921B680593E5
:1031C800002D11DC15E0013D069B002B03D105986D
:1031D8000670013005900134039800F053F8061C7E
:1031E800002D06DD411C04D0301C00F0DDF800285D
:1031F800E9D0301C0399FFF7D1FD069A002A1BD1AC
:103208000020059B187017E00124644214E0802216
:1032180041460A430095039807A90A23FFF7D2FD00
:10322800041C09E0802243461A430095039807A925
:103238001023FFF7C7FD041C002C08DA013417D14E
:103248000498002814D101235B42049310E0012361
:1032580041460B405A425341049AD2180492A14461
:103268007EE6C046CCCCCC0CFFFFFF7F9C3D000027
:10327800049809B03CBC90469946A246AB46F0BCBF
:1032880002BC084708B5031C0278002A06D0426829
:103298001078002806D001325A6005E0436800F033
:1032A80006F801E00120404208BC02BC0847184764
:1032B80070B5041C806800280AD0236862685D1C09
:1032C800AD1A6E1EB5416D422940934200D2C154D9
:1032D800E368002B07D020686268904203D2081C7C
:1032E800211C00F006F823680133236070BC01BC80
:1032F8000047184770B5151C4C1E07D40606360E35
:10330800281C311CFFF7D4FF013CF9D270BC01BC6A
:103318000047C04610B5C30606D42023840500D54F
:103328003023181CFFF7E6FF10BC01BC0047C0465D
:10333800031C413B002019229A4240417047C04675
:10334800031C613B002019229A4240417047C04645
:10335800031C303B002009229A4240417047C04676
:1033680038B5041C0D1CFFF7F3FF002802D0201C01
:10337800303811E0201CFFF7E3FF002802D0201CA2
:10338800573809E0201CFFF7D3FF002802D0201C83
:10339800373801E001204042A84201DB01204042C9
:1033A80038BC02BC0847C046021C093A0023042165
:1033B80091425B41203842424241181C10437047F9
:1033C800411C02780130002AFBD1401A7047C046E0
:1033D80010B582B0041C019100F010F88020204341
:1033E80000F0DAF801A800F0D7F800F00BF800F0C8
:1033F80007F8019802B010BC02BC08477047C046E5
:103408007047C046F8B54F464646C0B40F229046AE
:10341800042700F0ADF80409434618400A28F8D8F4
:103428008000514A13589F4600F0A2F8002C00D0A3
:1034380089E010E000F09CF83B1C28700135013C45
:10344800013B221C511E8A41002B02D0000A002A8F
:10345800F3D1002AEED1012000F09EF8D9E700F060
:1034680087F8002C14D0061C00250FE02D0A002C2C
:1034780004D03278120615430136013C013B002B7B
:10348800F4D1281C00F088F8002C01D03B1CEDE793
:10349800012000F081F8BCE700F06AF80126002C52
:1034A80056D117E000F064F83B1C29780135020674
:1034B800120E8A1A51424A4152421640013C013BBF
:1034C800221C511E8A41002B02D0000A002AECD18E
:1034D800002AE7D1301C00F05FF89AE700F048F8BE
:1034E800051C00F045F8002C04D028700135013C7B
:1034F800002CFAD1012000F04FF88AE700F038F8E4
:10350800012000F049F884E7012000F045F880E741
:1035180000F02EF8041C00F02BF8051C00F028F829
:10352800061C00F025F8814600F022F8031C281C30
:10353800311C4A4600F01AF800F02EF869E701201D
:1035480000F02AF80AE0051C00F012F83B1C74E7AA
:10355800051C00F00DF801263B1CA6E70CBC9046A4
:103568009946F8BC01BC00470C3F00002047C04604
:103578007847C0468FFCFFEA7847C046C9FCFFEA97
:103588007847C04683FCFFEA7847C046C5FCFFEA97
:103598007847C04683FCFFEA7847C0468DFCFFEABF
:1035A80009024300020100803209040000010202FE
:1035B800005E052400100105240101010424020213
:1035C8000524060001070581031000020904010013
:1035D800020A00005E070502024000000705820299
:1035E80040000000040309042A034700480049007A
:1035F800200045006C0065006300740072006F00D5
:103608006E006900630073002C0020004C004C0021
:1036180043000E0345004D00580020002000200004
:103628002A0342006F006F0054004C006F006100D5
:10363800640065007200200049006E007400650097
:10364800720066006100630065000000120100025C
:10365800020000089F1B0401000101020301000091
:10366800A10F0000D1180000D318000000000000CE
:103678000000000000000000000000000000000042
:103688000000000000000000000000000000000032
:103698000000000000000000000000000000000022
:1036A80000000000001000000020000000300000B2
:1036B80000400000005000000060000000700000A2
:1036C80000800000000001000080010000000200EE
:1036D80000800200000003000080030000000400D6
:1036E80000800400000005000080050000000600BE
:1036F8000080060000000700008007000090070017
:1037080000A0070000B0070000C0070000D00700B5
:1037180041726520796F7520737572652028592F5D
:103728004E293F0043616E63656C65642E00496EE7
:1037380076616C696420636F6D6D616E642E0076CE
:10374800322E302E34004F4B2E00555342697A6981
:103758000057616974696E672E2E2E004572726F6C
:10376800723A205468652075706C6F6164206661D8
:10377800696C65642E20506C65617365207472797C
:1037880020616761696E2E004572726F723A20542B
:1037980068652075706C6F616420697320636F724F
:1037A800727570742E0045726173696E672E2E2EC5
:1037B800004572726F723A205468657265206973A9
:1037C800206E6F206669726D77617265206F6E205A
:1037D800746865206465766963652E004572726F4A
:1037E800723A20546865206669726D776172652047
:1037F800697320636F72727570742E0053746172EE
:1038080074696E672E2E2E0068756E676E6172740D
:103818007175004572726F723A2054686520666946
:10382800726D776172652068617320756E65787056
:1038380065637465646C79206578697465642E20A5
:10384800506C6561736520636F6E746163742047A3
:1038580048492E0047484920456C656374726F6E6D
:103868006963732C204C4C4320426F6F746C6F61FA
:103878006465720D0A2D2D2D2D2D2D2D2D2D2D2DFF
:103888002D2D2D2D2D2D2D2D2D2D2D2D2D2D2D2D60
:103898002D2D2D2D004572726F723A2054686520C7
:1038A800646576696365206661696C656420746F18
:1038B80020696E697469616C697A652E20506C653F
:1038C80061736520636F6E74616374204748492E85
:1038D800000000002110422063308440A550C660DB
:1038E800E770088129914AA16BB18CC1ADD1CEE1B5
:1038F800EFF13112100273325222B5529442F7722C
:10390800D662399318837BB35AA3BDD39CC3FFF304
:10391800DEE36224433420040114E664C774A4443B
:1039280085546AA54BB528850995EEE5CFF5ACC554
:103938008DD55336722611163006D776F66695560B
:10394800B4465BB77AA719973887DFF7FEE79DD7A4
:10395800BCC7C448E5588668A7784008611802289B
:103968002338CCC9EDD98EE9AFF9488969990AA9F4
:103978002BB9F55AD44AB77A966A711A500A333A6B
:10398800122AFDDBDCCBBFFB9EEB799B588B3BBB44
:103998001AABA66C877CE44CC55C222C033C600CFB
:1039A800411CAEED8FFDECCDCDDD2AAD0BBD688D94
:1039B800499D977EB66ED55EF44E133E322E511E4B
:1039C800700E9FFFBEEFDDDFFCCF1BBF3AAF599FE4
:1039D800788F8891A981CAB1EBA10CD12DC14EF184
:1039E8006FE18010A100C230E320045025404670EA
:1039F8006760B9839893FBA3DAB33DC31CD37FE315
:103A08005EF3B1029012F322D23235421452776239
:103A18005672EAB5CBA5A89589856EF54FE52CD5E4
:103A28000DC5E234C324A014810466744764245489
:103A38000544DBA7FAB79987B8975FE77EF71DC7F4
:103A48003CD7D326F2369106B016576676761546D9
:103A580034564CD96DC90EF92FE9C899E9898AB944
:103A6800ABA94458654806782768C018E108823829
:103A7800A3287DCB5CDB3FEB1EFBF98BD89BBBAB54
:103A88009ABB754A545A376A167AF10AD01AB32A79
:103A9800923A2EFD0FED6CDD4DCDAABD8BADE89DA4
:103AA800C98D267C076C645C454CA23C832CE01CC9
:103AB800C10C1FEF3EFF5DCF7CDF9BAFBABFD98F34
:103AC800F89F176E367E554E745E932EB23ED10E19
:103AD800F01E0D0A000000008CB0F252849816AB5C
:103AE80092D5CF360BB211E84E290000702900009C
:103AF8007029000052290000702900007029000078
:103B08007029000056290000702900007029000063
:103B1800702900005C29000070290000622900005B
:103B28007029000070290000682900008C2D000011
:103B3800402A0000402A0000402A0000402A0000D5
:103B4800402A0000402A0000402A0000402A0000C5
:103B5800402A0000402A0000402A0000402A0000B5
:103B6800402A0000402A0000402A0000402A0000A5
:103B7800402A0000402A0000402A0000402A000095
:103B8800402A0000402A0000402A0000402A000085
:103B9800402A0000402A0000402A0000402A000075
:103BA800402A0000402A0000402A0000402A000065
:103BB800402A0000402A0000402A0000402A000055
:103BC8005E2A0000402A0000402A0000402A000027
:103BD800402A0000402A0000402A0000402A000035
:103BE800402A0000402A0000402A0000402A000025
:103BF800402A0000402A0000402A0000402A000015
:103C0800402A0000402A0000402A0000402A000004
:103C1800402A0000402A0000402A0000402A0000F4
:103C2800402A0000402A0000402A0000402A0000E4
:103C3800402A0000402A0000402A0000402A0000D4
:103C4800402A0000402A0000402A0000402A0000C4
:103C5800402A0000402A0000402A0000402A0000B4
:103C6800402A0000402A0000402A0000402A0000A4
:103C7800402A0000402A0000402A0000402A000094
:103C8800402A0000402A0000402A0000342B00008F
:103C9800402A0000402A0000402A0000402A000074
:103CA800402A0000402A0000402A0000402A000064
:103CB800402A0000402A0000682A00007C2B0000EF
:103CC800402A0000402A0000402A0000402A000044
:103CD8007C2B0000402A0000402A0000402A0000F7
:103CE800402A00009A2A00005A2B0000162B0000D8
:103CF800402A0000402A0000BE2A0000402A000096
:103D08006E2B0000402A0000402A00003A2B0000D9
:103D1800162C0000C82C0000C82C0000C82C00007D
:103D2800C82C0000C82C0000C82C0000C82C0000BB
:103D3800C82C0000C82C0000C82C0000C82C0000AB
:103D48000E2C0000C82C0000C82C0000C82C000055
:103D5800C82C00000E2C0000C82C0000C82C000045
:103D6800C82C0000C82C0000C82C0000042C00003F
:103D7800162C0000C82C0000C82C0000C82C00001D
:103D8800C82C00000E2C0000C82C0000C82C000015
:103D9800162C0000783000007832000078320000DD
:103DA8007832000078320000783200007832000063
:103DB8007832000078320000783200007832000053
:103DC8007832000078320000783200007832000043
:103DD8007832000078320000783200007832000033
:103DE8007832000078320000783200007832000023
:103DF8007832000078320000783200007832000013
:103E08007832000078320000783200007832000002
:103E180078320000783200007832000078320000F2
:103E280078320000783200007832000078320000E2
:103E380078320000783200007832000078320000D2
:103E480078320000783200007832000078320000C2
:103E580078320000783200007832000078320000B2
:103E68002C320000783200007832000078320000EE
:103E78007832000078320000783200007832000092
:103E8800783200007832000078320000A630000056
:103E98000E310000783200007832000078320000DD
:103EA80078320000243100007832000078320000B7
:103EB80078320000783200003A31000068310000A2
:103EC8007E31000078320000783200009431000022
:103ED8007832000016320000783200007832000094
:103EE8002C3200003031323334353637383961629C
:103EF8006364656630313233343536373839414298
:103F0800434445463034000066340000E434000081
:103F1800043500001035000046350000A0340000CC
:103F28001A3400001A340000183500006435000007
:0400000300000410E5
:00000001FF
